:100000000C945A100C9482100C9482100C94821050
:100010000C9482100C9482100C9482100C94821018
:100020000C9482100C9482100C9493120C9405136F
:100030000C9482100C9482100C9482100C948210F8
:100040000C9482100C943E170C9482100C94821025
:100050000C9482100C9482100C9482100C9406164E
:100060000C9482100C9482100C9482100C948210C8
:100070000C9482100C9482100C9482100C948210B8
:100080000C9450160C9482100C9482100C948210D4
:100090000C9482100C9482100C9482100C94821098
:1000A0000C9482100C9482100C948210F0F89C8EA8
:1000B0008783878E9CF8F00000FEFF030303030391
:1000C000070EFCF80000FEFF0303030303070EFC0A
:1000D000F80000FFFF00000000000000FFFF00002C
:1000E000FEFF8383838383C7EE7C380000F8FC0E19
:1000F00007030303070EFCF800003F7FE0C0808089
:10010000C0E07F3FFFFF01010101010101FFFF008E
:1001100000FFFF0C0C0C0C1C3E77E3C100007FFFBE
:10012000C0C0C0C0C0E0703F1F00001F3F70E0C0F3
:10013000C0C0E0703F1F00007FFFC1C1C1C1C1E36B
:10014000773E1C00001F3F70E0C0C0C0E0703F1F42
:10015000000000000001FFFF01000000D5F08D1439
:10016000A1C881CFD9F1AF20000A53636F72650A2D
:100170000A000A4E65770A48692D53636F7265213C
:100180000A0A0047616D65204F7665720A0000001B
:10019000000000000000000000000000000000005F
:1001A00000000000000000000000FF000000000050
:1001B000000000FF000000000000030F3AE6FF000F
:1001C00000000000000000FF00000000FE0301002E
:1001D0000000FF0000000000000000FF0000000021
:1001E000000000000000FF0000000000000000FF11
:1001F00000000000000000000000FF000000000000
:10020000000000FF000000000000000000000000EF
:1002100000000000000000000000000000000000DE
:1002200000000000000000000000FF0000000000CF
:10023000000000FF00000000000000000000FF00C0
:1002400000000000000000FF063C080C0704040446
:10025000040C1B78C0000000000000FF000000003C
:10026000000000000000FF0000000000000000FF90
:1002700000000000000000000000FF00000000007F
:10028000000000FF0000000000000000000000006F
:10029000000000000000000000000000000000005E
:1002A00000000000000000000000FF00000000004F
:1002B000000000FF00000000000000000080FF00C0
:1002C00000000000000000FF000000004040C040AF
:1002D000C098900001070408183060FF000000007B
:1002E000000000000000FF0000000000000000FF10
:1002F00000000000000000000000FF0000000000FF
:10030000000000FF000000000000000000000000EE
:1003100000000000000000000000000000000000DD
:1003200000000000000000000000FF0000000000CE
:10033000000000FF00000000000000E0BCC7FF005C
:1003400000000000000000FFC000404040C080816D
:100350000101010030F8F8840060E0E1E3EEF8E824
:100360001810307050D0FF0000000000000000FFA7
:1003700012123321216141418181FF000000000000
:10038000000000FF24040C08080808080808000002
:10039000000000000000000000000000000000005D
:1003A00000000000000000000000FF00000000004E
:1003B000000000FF0000000000C0701F0707FF00E2
:1003C00000000000000000FF01038606060E0E0F6D
:1003D0000F0EFE0E060707070F0C08FDFF27010092
:1003E000101030000000FF0000000000000000FFBF
:1003F00000000000000000000000FF0000000000FE
:10040000000000FFE8E8D8B8E848D8B8307000002D
:1004100000000000000000000000000000000000DC
:1004200000000000000000000000FF0000000000CD
:10043000000000FF00000000C0FF00000080FF007F
:1004400000000000000000FF18040200000000048B
:100450000010FF0000000000000000FF03060C0C6D
:100460000C1C32618000FF0000000000000000FF53
:1004700000000000000000000000FF00000000007D
:10048000000000FF81030343416373F3F97C000024
:10049000000000000000000000000000000000005C
:1004A00000000000000000000000FF00000000004D
:1004B000000000FF000000FFFFFF000000070F1C0E
:1004C0001C1818383010101F101010101030202079
:1004D00020203F20202060404040407F4242424058
:1004E0004040A0603F00FF0000000000000000FF4F
:1004F000080808080808080C0C0CFF0000000000A1
:10050000000000FF01010101406020303333000092
:1005100000000000000000000000000000000000DB
:1005200000000000000000000000FF0000000000CC
:10053000000000FF000000000F1810202020E02025
:1005400020202020202020F010101808080808087B
:100550000808F80808080808080818F01010101E05
:100560007DDBF9F3327EFF0000000000000000FF99
:1005700010302020202020202020FF00000000003C
:10058000000000FF18383838280818100010FF0144
:1005900079157901FFFE82AAD6FE00010101010151
:1005A000010100000000000000FE86EA86FEFF0157
:1005B0007D552901FF00000000000001010101013B
:1005C0000101C040C08000000000000000000000E9
:1005D0000000008080C04060301098C8ECA464C463
:1005E000CC9890B0A0A020B0DFE971B7ACA898F08B
:1005F00000000000000003060C19133226242424F6
:10060000242632121311111118080A08091B37EF9A
:1006100085192B1680F0F95B4980E1390C0603013E
:1006200000000000000000000000000000000000CA
:1006300000000000000000000000000000000000BA
:100640000000001E13103062C78C99F101010000F8
:10065000000000000000000000000000000000801A
:10066000000000000000000000000000000000008A
:1006700000008080C0E060301058983830606040E2
:100680004040C04020168E485050600000000000DE
:100690000000000103060C0C1818181818180C0C90
:1006A0000C0E0E0E07070507060408107AE6D4E9BB
:1006B0007F0F06A4B67F1E060301000000000000A5
:1006C000000000000000000000000000000000002A
:1006D000000000000000000000000000000000001A
:1006E0000C0F0F1D387060000000000000000000BB
:1006F00000000000000000000000000000000000FA
:10070000000000000000000080C0406020B0909019
:10071000D0D0903020A020B7DDE973B6ACA898F017
:1007200000000000000000000000000000000000C9
:1007300000F0903060406030188CC643E1E46223E2
:10074000474F6F3DB396C9637356E53198E63F0155
:100750000000000000000000000000000000000099
:10076000000000000000010302020203010100F08A
:100770009F80C07E02030101010000000000010112
:100780000100000000000000000000000000000068
:100790000000000000000000000000000000000059
:1007A0000000000000008080C0406060202060C029
:1007B000C040C04022168C4850506000000000002D
:1007C000000000000000000000000000000060C009
:1007D000808080C0E070383C1E1B9DDCB8B090C2A9
:1007E0004C69361C0C291ACE671900000000000065
:1007F00000000000000000000000000000000000F9
:10080000000000000101010000000000607F3F01C6
:1008100001000000000000000000000000000000D7
:1008200000000000000000000000000000000000C8
:1008300000000000000000186CD6AAD6AA562AB400
:10084000A830E0000040A0905048241413090A0B7F
:100850000B0504020300000000000000000000007F
:100860000000000000000000000000001864922951
:10087000552955A9D54A54C810E040A05068A8B4DD
:100880005A2B2C161514140A0B0504030000010141
:100890000000000000000000000000000000000058
:1008A000000000008060361EA0A040808000000094
:1008B00000003C242231383C0804050404080809DF
:1008C0000600000000000000000000000000000022
:1008D00000000000000000000080609EC9E15E5042
:1008E000A04040800000003C425A5D4E4743370B19
:1008F0000A0B0B1717160906000000000000000085
:1009000000000000000000000000FF0101010101E3
:1009100001010101010101010101010101010101C7
:1009200001010101010101010101010101010101B7
:10093000FF0F080808080808080808080808080839
:100940000808080808080808080808080808080827
:10095000080808080808080F00C04070109848AC44
:1009600044A454A454A454A454A40CC8C8D810B08B
:1009700020A0401E13101A090A090A090A09088D45
:10098000E0F9F8FDFCFEFF0FC7300C03010000008A
:10099000000000000000000000000373FFFFFFFFE5
:1009A000BF1900010000000000000000000000006E
:1009B0000000008080C0E0EFFF7F7F1F000000008C
:1009C00000000000000000000000000000033F3FA6
:1009D0003F37310000000000000000000000000070
:1009E000000000000080E0388C47A955A852A55BA4
:1009F000261CB08080800000000000000000000085
:100A0000FF8014AA552A95CAE5F2F9F8FCFFEF0F0A
:100A100083C0C00000000000000000000F784241C9
:100A200078030FFFFFFFFFFFC707070301010C005B
:100A3000000000000000707C1C1818383878797F9E
:100A40003F0F071FFFFEF000000000000000000045
:100A50000000000000000000000000000000000195
:100A6000073F38303000000000000000C060B05880
:100A7000A848A84CA652AA52AA12AA92AA823A023E
:100A8000FE0000C0788E53A9D46A252A252A350293
:100A9000F1FAF9F8FCFFCF0703F8000F000003029A
:100AA0000203010000000000000070FFFFFFFFDFF5
:100AB00007060606760000000000000000E0F83897
:100AC0001818383038383F3F3F0F9FFFF8000000BC
:100AD0000000000000000000000000000000000016
:100AE0000000000000033F3F202000000000C06025
:100AF00020B0509848AC44A456A252AA52A216C4A0
:100B0000E4E4EC0828C818E00F090C06020202020F
:100B1000020242E2F2F8FCFEFEFEFFFF036318034E
:100B200001020100000000000000000000000107B9
:100B30007FFFFFFFEF8F0C0C0000000000000000A3
:100B400000000000003C3E0E0C0CEEFE3F1F0F0F9D
:100B50000F00000000000000000000000000000086
:100B6000000000303F3F3120200000000000000066
:100B70000000000000000000000000E0301848AC59
:100B8000C446D28A1A8ADAC2D6044C9830E00000F1
:100B9000000000000000C1E1F1F93938F8F8FCFC70
:100BA000FFFF87172015AA200FF80000000004049B
:100BB00000070F0F0600F0FFFFFFDF870F0F0E0685
:100BC0000707030003000000181E0F07070E0E1E84
:100BD0001E1C3F3F0F0FFFFEE00000000000000062
:100BE0000000000000000000000000000000000005
:100BF0000000073F3C303000000000000000000013
:100C000070584C4454C494A454244C08C8C8D810F8
:100C100050B060C0800000000000000000000080B4
:100C2000C0E0F1F9FCFCFEFFE707201D1A0A0409E9
:100C30000F00000000000000002011030FFFFFFF65
:100C4000FF8F0F0F0F0E0F070000000000000000C5
:100C5000003C3E1E0E0E0C0C1C1F1FFFFFF8000078
:100C60000000000000000000000000000000000084
:100C700000000000000000073F3C30302000000072
:100C8000000000008080E060B050B858A858A85814
:100C9000A858A858F0303020E040C04080000C0F29
:100CA0000506050605060506C7721F0607020301AD
:100CB00000F038CF330C06010000000000000000F7
:100CC00000000007FC8C0000000040E63F06010029
:100CD000000000000000000000000080C040603004
:100CE0001F10008080E03F000000000000000000B6
:100CF000000000000000073C000000080E3B01005F
:100D000000000000000000000000000000000000E3
:100D100000C070B856AA57AD5AA4D8E04040404031
:100D2000C0000000000000000000007FEB55AAD5C5
:100D30006A351A0D0607030010F07C3720E000002A
:100D400000000000000000073D3E071CF00000000E
:100D5000000038E8880C060E130E0000000000F8B2
:100D60008E82E2266444C4878680C07038E0000129
:100D70000FF800000000000000000000000000006C
:100D80000000000000000000030E3800070C0838C7
:100D9000000000000000008040A050B050B058ACEF
:100DA00054AC54EC546C547CC4FC000000008070C3
:100DB000AC562B151A151A150AFD0E050607030069
:100DC00030F8FC07FF0000000001010000000000F7
:100DD000000000F88F0000000020F88909F989FF61
:100DE000000000000000F01C04C46464444C44474C
:100DF000404040F0600007FC0000000000000000E0
:100E00000001010101000000000000000000073C9B
:100E100000001F10300000000080C040A060B050F3
:100E2000B858A85CAC54AC5CE838181810F0D03056
:100E3000E000000603010101010101E1B1190D0704
:100E4000030101010000FC9C671C0601000000007A
:100E500000000000000000030EF880000000107089
:100E6000D3131F00000000000000000000007E43BC
:100E7000417193F31101C0603010101F0000000099
:100E8000000000000000000000000000380F00001B
:100E90000E1B1030000000000000000000000000E9
:100EA000000000000000C0E0B05038382C74E4743A
:100EB000243C28F8B060C00000000000000000E002
:100EC00030180C04C4C404060203000078E8DFEA0A
:100ED00055DFF0000000000E8A8A8F98901019FFED
:100EE0000F0000002078D010111908080C0700002E
:100EF000003C27213018181131212163404070F047
:100F000000011FF0000000000000000000000000D1
:100F100000000000000000000000010F3800030E78
:100F20000838000000000000000000203038283899
:100F30006858A8D8B0F0303020E0A0408000000011
:100F40000000000000000000C06030180C06030321
:100F5000010018F8DFA2A5950B06000000000000B4
:100F60000000305B2E3CF00000000070D01010112B
:100F700010180F000000000000007E434161311195
:100F800013332320E0000007FC00000000000000F5
:100F90000000000000000000000000000000000150
:100FA0000F3800030E081830000000000000000099
:100FB000000000000000FC02F90402010000000033
:100FC0000000000000000000000000000000FF0022
:100FD000FF00000000000000000000000000000012
:100FE000000000000000FF00FF0000000000000003
:100FF0000000000000000000000000000000FF00F2
:10100000FF000000000000000000000000000000E1
:10101000000000000080FF80FF8000000000000052
:1010200000000000000000000000000000FB8480C1
:1010300084FB000000000000000000000000000031
:101040000000000001010101010101000000000099
:101050000000000000000000000000000000000090
:101060000000000000000000000000000000000080
:101070000000000000000000000000000000000070
:101080000000000000000000000000000000000060
:101090000000000000000000000000000000000050
:1010A0000080000000408000008000000000000080
:1010B00000000000000038E82A2C2F2E2D2C2F2EA7
:1010C0002FE82C2E2E2F2C2CE8380000000000FFDB
:1010D00022222222223E22222223E22222223E22F7
:1010E000FF000000000000010101010101010101F8
:1010F00001010101010101010100000000000000E7
:1011000000000000000000000000000000000000DF
:1011100000000000000000000000000000000000CF
:1011200000000000000000000000000000000000BF
:1011300000000000000000000000000000000000AF
:101140000000000000000000C0B860C01AEE98F077
:10115000BC76F0C8C020008000000000000038EA23
:10116000282F2F2F2FEF2F2E2F2B2D2F2E2F2F2CE1
:10117000E8380000000000FF223E222222E3222263
:10118000223E222222223E22FF0000000000000117
:10119000010101010101010101010101010101013F
:1011A00001000000000000000000000000FE03FD40
:1011B00006FB0D0603000000000000000000000018
:1011C0000000000000FF00FF00FF00000000000022
:1011D00000000000000000000000000000FF00FF11
:1011E00000FF000000000000000000000000000000
:1011F0000000000000FF00FF00FF000000000000F2
:10120000000000000000000000000000C07F007F20
:10121000007FC0000000000000000000000000008F
:1012200000000080FF047B7F7B04FF800000000043
:1012300000000000000000000000000302020202A3
:101240000202020300000000000000000000000095
:10125000000000000000000000000000000000008E
:10126000000000000000000000000000000000007E
:10127000000000000000000000000000000000006E
:10128000000000000000000000000000000000005E
:101290000000000000000000C040C080E0A060C06E
:1012A000C040C0008080800000000000007CC417A7
:1012B000D5D3D0D1D2D3D0D1D017D3D1D1D0D3D2CE
:1012C00016C47C000000FF00DDDDDDDDDDC1DDDDFD
:1012D000DDDC1DDDDDDDC1DD00FF000000000302FF
:1012E00002020202020202020202020202020202DE
:1012F00002030000000000000000000000000000E9
:1013000000000000000000000000000000000000DD
:1013100000000000000000000000000000000000CD
:1013200000000000000000000000000000000000BD
:10133000000000000000000000000000000000E0CD
:101340003C449C3FE511670E43890F343CD0F0408C
:10135000C0000000007CC415D7D0D0D0D010D0D1B0
:10136000D0D4D2D0D1D0D0D317C47C000000FF009D
:10137000DDC1DDDDDD1CDDDDDDC1DDDDDDDDC1DDB2
:1013800000FF000000000302020202020202020249
:101390000202020202020202020300001190909176
:1013A0000180FF0C0C0C0C0808FF8F0C0C0C0C0CB3
:1013B0000C0C0C0C08FFCF0C0C0C0C0808FF9191C6
:1013C0009181FF00000000000000000000FF8888FD
:1013D00088080008FF606060604040FF7F606060D8
:1013E00060606040404040FF7F606060604040FF60
:1013F00088880808FF00000000000000000000FFCF
:10140000042024042004FF808080800000FFFE80F0
:10141000808080808080808000FFFF80808080804E
:1014200000FF20240404FF00000000000000000072
:1014300000FF8989888989E88989898F898989F95B
:101440008989898D898189898989F9898F8989899A
:10145000898981898889B988FF404040404040405F
:10146000404040FF2424242724243C2424242624F0
:101470002C24242724243C2424252424242C242400
:101480002724243C2424272424247F404040404017
:1014900040404040407F000000000000000000008D
:1014A000000000000000000000000000000000003C
:1014B000000000000000000000000000000000002C
:1014C000000000000000000048692D53636F726542
:1014D0003A000000000000000000000000000000D2
:1014E000000000001FE0077FFEFCF9F9E2E2ECC813
:1014F000D090A020C000000000000000000000000C
:10150000000000000000000000000000804020906B
:10151000C8E8E4F4F2F9F28428D0000000000000EA
:1015200000000000000000000000000000000000BB
:1015300000000000000000000000000000000000AB
:10154000000000000000000000000000000000009B
:10155000000000000000000000000000000000008B
:10156000000000000001060830479F3F7FFFFFFF9B
:10157000FFFFFFFEFCF9F2C498204080000000004D
:101580000000000080406010C8E4F2F9FCFEFFFF9C
:10159000FFFFFFFF7F1FCFE1DCC3C0C0C0C0000062
:1015A000C0C0C0C0C0C0C0C0C0C0C0C0000000003B
:1015B000C0C0C0C0C0C0C0C0C0C0C0C0000000002B
:1015C000C0C0C0C0C0C0C0C0C0C0C0C0000000001B
:1015D000000000000000000000000000000000000B
:1015E000000000000000000000000001060833C7F2
:1015F0001F7FEFFFFF9FB7EFFFFFFEF8F3E4E8E880
:10160000E4F4F2F9FCFEFFFF7FFF7F3FBFFF1FCF37
:10161000231B09646667666666666666660000FC8C
:10162000FFFFFFE7E1E1E1FFFFFFFF03000000F83C
:10163000FFFFFF07030303FFFFFFFF07000000F8A2
:10164000FFFFFF07030303FFFFFFFF07000000008A
:1016500000002C042018002000000820A010000822
:101660001080420080000000000000000000000721
:10167000887003FFFF7F7F7FFDBFFF3FFF7FBB8F32
:10168000BF7F3B5FFFF3FCF0FE3E1FC33B0804033C
:1016900020000000000006060606E6E60600F8FF49
:1016A000FFFF0F01031FFFFFFFF901000000F0FF24
:1016B000FFFFFFE0E0E0F8FFFFFF0F000000F0FF9A
:1016C000FFFFFFE0E0E0F8FFFFFF0F000000000079
:1016D000000064C02000005000880201205020005B
:1016E000000080004000000000000800000000F83A
:1016F0000770FFFFFEF0C0E8F8FFFF7FBFFDFFDED1
:10170000FFA07CF8F08080C0E005F0BFB0B0B0B0C2
:10171000B0300000F0F0F0F0707070F0F0F0F1F127
:1017200001010000F0F0F1F101010000F0F0F1F131
:1017300001010101F1F1F1F1F1F1F0F0F0F0F1F15D
:10174000010101010101010101010000000000008F
:10175000000074F4F4E4E8E8E8C8E8E8C8CAE8E996
:10176000C8D0D0D1D091D0D1D2D012D050905F80FB
:10177000F0FFBF7FEBCF9FFF9FF771BDBF7F7F6FF4
:101780007F7DBCF2E71F07E3180611199999999913
:10179000990000FFFFFFFF79F8F8F8FFFF7F7F0057
:1017A000000000FEFFFFFF03000000FFFFFFFF013E
:1017B000000000FEFFFFFF03000000FFFFFFFF012E
:1017C0000000000000000000000000000000000019
:1017D00080009F69B6695E37875F87EF573F8B3719
:1017E0004B07150FC5ABD54E75A6605A8CF2ADF4FC
:1017F000507FBFFEF5CFBBFF7FFFFEF8E0C0C0C04B
:10180000C060F89C0FC03E01000080000101393922
:1018100001007E7F7F7F030000077F7F7F7E0000C7
:1018200000007C7F7F7F7F7878787E7F7F7F0300DA
:1018300000007C7F7F7F070000007E7F7F7F0300AA
:10184000000000000000000002000020000801006D
:1018500000012BD509EA57681B2D8A3711001204A5
:1018600090C0E85AB6EABFE5FAF7D8FFF4EBBEFF3E
:10187000F7FDEBFEFFFFFE570107010304350203EE
:10188000156BBFFF400FF00000804020D08020206B
:101890006008B040444A1480220810002008240246
:1018A00028042200100008020000201000000000A0
:1018B0000400000004000000000000000000000020
:1018C000006200040000000005000800000124057B
:1018D000100063726169742E6E65740040637261FA
:1018E000697400486F6C6D6573004A6F6E6174684F
:1018F000616E00458A15AA15AAD56A342821321DC1
:101900000A0C06030207022341A0418040814020C7
:10191000804080402008C77DA255A251A815884468
:10192000A251AA54A8518205FF0000418080008086
:10193000E0F0F0F0F0E060606068EDE4E3E0E061CA
:1019400072E102E1321AAF1188548A452A059245A4
:10195000A241A055AA55AA55BFE0000000003CFED8
:10196000FFFFFF1DEC3637F7F7EE1FFF3FDF2E3787
:10197000F6EE1C037E55CAC5A251A854AA552A15D5
:101980008A452251A254A055FEC3BC66400038DFF0
:101990007FBFFFFFFE7D7D7DFDFE3F7FFFF06D1D64
:1019A000BDFEFFE0833FC07FA255A2512804A25193
:1019B000A854AA11A215A2C56A4563416B5E78714D
:1019C000A64B8D979C38312306464D4D6D727F6F27
:1019D0001F370F1DCBE07F556A4540C08AC56AB5E9
:1019E000DAEDCA3DCEF3FDFEF8877FFFFFFFFFC0B3
:1019F000BFBEBDDB57A7CFB78BFAF676A6CA76EA8D
:101A00009C5FDFC0FEFEFFFFFFFF0FB6B9FBF8F3E0
:101A1000F7FFF801020408102040800000000000D9
:101A20003E5B4F5B3E3E6B4F6B3E1C3E7C3E1C184C
:101A30003C7E3C181C577D571C1C5E7F5E1C0018AA
:101A40003C1800FFE7C3E7FF0018241800FFE7DB9E
:101A5000E7FF30483A060E2629792926407F0505FA
:101A600007407F05253F5A3CE73C5A7F3E1C1C0837
:101A7000081C1C3E7F14227F22145F5F005F5F06FC
:101A8000097F017F006689956A606060606094A24A
:101A9000FFA29408047E040810207E201008082A63
:101AA0001C08081C2A08081E101010100C1E0C1E02
:101AB0000C30383E3830060E3E0E060000000000A6
:101AC00000005F00000007000700147F147F14244B
:101AD0002A7F2A12231308646236495620500008D0
:101AE000070300001C2241000041221C002A1C7F29
:101AF0001C2A08083E080800807030000808080802
:101B000008000060600020100804023E5149453E74
:101B100000427F400072494949462141494D3318EE
:101B200014127F1027454545393C4A494931412126
:101B30001109073649494936464949291E0000140A
:101B40000000004034000000081422411414141452
:101B500014004122140802015909063E415D594E04
:101B60007C1211127C7F494949363E414141227F16
:101B70004141413E7F494949417F090909013E41AF
:101B80004151737F0808087F00417F410020404198
:101B90003F017F081422417F404040407F021C02E9
:101BA0007F7F0408107F3E4141413E7F09090906BD
:101BB0003E4151215E7F0919294626494949320390
:101BC000017F01033F4040403F1F2040201F3F4016
:101BD00038403F63140814630304780403615949CF
:101BE0004D43007F41414102040810200041414122
:101BF0007F04020102044040404040000307080007
:101C000020545478407F2844443838444444283889
:101C10004444287F385454541800087E090218A4FC
:101C2000A49C787F0804047800447D400020404054
:101C30003D007F1028440000417F40007C04780470
:101C4000787C080404783844444438FC1824241868
:101C500018242418FC7C0804040848545454240410
:101C6000043F44243C4040207C1C2040201C3C403D
:101C700030403C44281028444C9090907C4464545C
:101C80004C4400083641000000770000004136084F
:101C90000002010204023C2623263C1EA1A161127F
:101CA0003A4040207A3854545559215555794121AC
:101CB00054547841215554784020545579400C1E95
:101CC000527212395555555939545454593955543D
:101CD00054580000457C410002457D420001457C8E
:101CE00040F0292429F0F0282528F07C545545009F
:101CF0002054547C547C0A097F4932494949323284
:101D000048484832324A4848303A4141217A3A42BA
:101D1000402078009DA0A07D39444444393D404096
:101D2000403D3C24FF2424487E4943662B2FFC2F52
:101D30002BFF0929F620C0887E09032054547941DD
:101D40000000447D413048484A32384040227A0001
:101D50007A0A0A727D0D19317D2629292F28262914
:101D600029292630484D4020380808080808080866
:101D700008382F10C8ACBA2F102834FA00007B00A6
:101D80000008142A142222142A140895002200950F
:101D9000AA005500AAAA55AA55AA000000FF0010E3
:101DA0001010FF00141414FF001010FF00FF10109B
:101DB000F010F0141414FC001414F700FF0000FFDE
:101DC00000FF1414F404FC141417101F10101F103B
:101DD0001F1414141F00101010F0000000001F103A
:101DE0001010101F10101010F010000000FF101045
:101DF00010101010101010FF10000000FF14000051
:101E0000FF00FF00001F10170000FC04F41414175B
:101E100010171414F404F40000FF00F71414141441
:101E2000141414F700F7141414171410101F101FB3
:101E3000141414F4141010F010F000001F101F0000
:101E400000001F14000000FC140000F010F010103F
:101E5000FF10FF141414FF141010101F00000000D6
:101E6000F010FFFFFFFFFFF0F0F0F0F0FFFFFF00CA
:101E700000000000FFFF0F0F0F0F0F3844443844DD
:101E80007C2A2A3E147E02020606027E027E02633D
:101E9000554941633844443C04407E201E200602DC
:101EA0007E020299A5E7A5991C2A492A1C4C7201B9
:101EB000724C304A4D4D303048784830BC625A46FA
:101EC0003D3E494949007E0101017E2A2A2A2A2AEB
:101ED00044445F444440514A444040444A514000D5
:101EE00000FF0103E080FF000008086B6B0836125A
:101EF000362436060F090F060000181800000010DF
:101F000010003040FF0101001F01011E00191D17C4
:101F100012003C3C3C3C000000000000000000249B
:101F20000027002A002D00300000000000250028B6
:101F3000002B002E003100040802011040804010E8
:101F400020408040800802040180402010020110DF
:101F5000801020404020040404040403040502020D
:101F60000202040302020202060606060606040432
:101F7000020202040406011501260137014A015D2F
:101F800001720188019F01B801D201EE010B022A02
:101F9000024B026E029302BA02E40210033F037086
:101FA00003A403DC03170455049704DD0427057517
:101FB00005C80520067D06E0064907B8072D08A9D3
:101FC000082D09B9094D0AEA0A900B400CFA0CC019
:101FD0000D910E6F0F5A1053115B1272139A14D495
:101FE0001520178018F519801B231DDE1EB420A6AE
:101FF00022B524E4263429A72B402E0031EA3300F1
:1020000037453ABC3D68414C456B49C84D68524F15
:1020100057805C006210111213151617181A1C1D38
:102020001F21232527292C2E3134373A3E4145499B
:102030004E52575C62686E757B838B939CA5AFB9DB
:10204000C4D0DCE9F7080B00020202010009040019
:102050000001020200000524001001052401010115
:102060000424020605240600010705810310004030
:1020700009040100020A00000007050202400000F6
:10208000070583024000000403090412010002EF67
:1020900002014041233680000101020301417264C4
:1020A00075696E6F204C4C430041726475626F79A4
:1020B0000000612311241FBECFEFDAE0DEBFCDBFE9
:1020C00011E0A0E0B1E0E4E2F9E402C005900D9275
:1020D000AE33B107D9F725E0AEE3B1E001C01D9200
:1020E000A43FB207E1F710E1CAE5D0E104C02197AF
:1020F000FE010E948524C935D107C9F70E94F71C4B
:102100000C9490240C940000409172015091730142
:10211000209170013091710142175307B4F49091EE
:10212000E8009570E1F39091E80092FD19C080936A
:10213000F100809172019091730101968F7399273C
:10214000892B19F48EEF8093E800809172019091B1
:1021500073010196909373018093720181E0089559
:1021600080E00895DF92EF92FF920F931F93CF9339
:10217000DF93D82E8A017B01E40EF51EEB01CE150C
:10218000DF0571F0D7FE03C0FE01849101C0888194
:102190000E94841021968111F2CF8FEF9FEF01C032
:1021A000C801DF91CF911F910F91FF90EF90DF90C9
:1021B0000895615030F02091F100FC0120830196D8
:1021C000F8CF289884E6809375010895CF92DF9226
:1021D000EF92FF920F931F93CF93DF936C017A01DD
:1021E0008B01C0E0D0E0CE15DF0589F0D8016D91FC
:1021F0008D01D601ED91FC910190F081E02DC60199
:102200000995892B11F47E0102C02196ECCFC701FC
:10221000DF91CF911F910F91FF90EF90DF90CF90C2
:102220000895CF93DF931F92CDB7DEB76983DC01AA
:10223000ED91FC910280F381E02D41E050E0BE0180
:102240006F5F7F4F09950F90DF91CF91089583E0E5
:102250008093E9008091F200882319F08AE380934B
:10226000E8000895FC018485958597FD0BC09FB714
:10227000F89482E08093E9008091F2009FBF90E0A3
:10228000019608959FB7F89482E08093E9008091C9
:10229000F2009FBF90E008953FB7F89480916C01E1
:1022A00090916D01A0916E01B0916F0126B5A89B30
:1022B00005C02F3F19F00196A11DB11D3FBFBA2FD8
:1022C000A92F982F8827820F911DA11DB11DBC0138
:1022D000CD0142E0660F771F881F991F4A95D1F7FD
:1022E0000895CF92DF92EF92FF921F93CF93DF93E7
:1022F000E82FF0E0EC5EFE4F1081E62FF0E0603357
:1023000030F4EB5EFF4DE491CE2FD0E006C0EE0F2F
:10231000FF1FEB5EF04EC591D4916E01E12CF12CC4
:1023200060E074E284EF90E0A70196010E940E2421
:10233000DA01C9010197A109B109009721E0A207BB
:10234000B10578F060E970ED83E090E0A7019601B7
:102350000E940E24DA01C9010197A109B10923E005
:1023600001C021E01130C9F0133051F530919100D6
:10237000387F232B209391009093990080939800AD
:10238000D0936901C093680181E0809367018091D7
:10239000710082608093710013C030916A01311125
:1023A0000FC030918100387F232B209381009093C0
:1023B00089008093880080916F00826080936F0015
:1023C000DF91CF911F91FF90EF90DF90CF90089514
:1023D000E82FF0E0EC5EFE4F8081813019F0833011
:1023E00089F0089580916A01811122C080916F0067
:1023F0008D7F80936F0090915401E0915201F09194
:1024000053010CC01092670180916601811110C0C8
:1024100090916401E0916201F09163018081282F25
:1024200030E0892F90E080959095822393238083DC
:10243000089580914101089508950E948B240F937F
:102440001F93CF93DF931F92CDB7DEB782E08983CE
:1024500042E450E065E470E280E80E94B2100E941D
:10246000E31CDC0112960D911C91139701151105C7
:1024700069F0D801ED91FC910280F381E02DBE015D
:102480006F5F7F4FC801099597FF07C089810F9043
:10249000DF91CF911F910F910895F801008511856B
:1024A000E5CF0F931F93CF93DF931F92CDB7DEB786
:1024B0008C01FC018485958597FF0EC0CE010196A5
:1024C0000E94B91C019719F4298130E002C02FEF56
:1024D0003FEFF80135872487F801848595850F90B3
:1024E000DF91CF911F910F910895CF93DF931F92AA
:1024F000CDB7DEB7FC018485958597FD05C02FEF2C
:102500003FEF358724870BC0CE0101960E94B91C8E
:10251000019719F4898190E002C08FEF9FEF0F902F
:10252000DF91CF9108951F920F920FB60F92112451
:102530008F939F938091E1009091E100937F90931E
:10254000E10083FF0FC01092E90091E09093EB004F
:102550001092EC0092E39093ED001092760198E0D7
:102560009093F00082FF20C093E09093E900909157
:10257000F200992319F09AE39093E8009091740186
:10258000992339F09091740191509093740199239B
:1025900089F190917501992339F0909175019150CD
:1025A00090937501992341F184FF10C08091E2005E
:1025B0008E7E81608093E2008091E1008F7E809327
:1025C000E10080913F018E7E806111C080FF16C0C6
:1025D0008091E2008E7E80618093E2008091E10034
:1025E0008E7E8093E10080913F018E7E816080939A
:1025F0003F0104C05D9ACDCF289AD6CF9F918F918D
:102600000F900FBE0F901F9018951F920F920FB64C
:102610000F921124CF92DF92EF92FF920F931F93AC
:102620002F933F934F935F936F937F938F939F93DA
:10263000AF93BF93EF93FF93CF93DF93CDB7DEB705
:102640006C97DEBFCDBF1092E9008091E80083FF58
:10265000EDC168E0CE0145960E94D91082EF8093CB
:10266000E8008D8987FF05C09091E80090FFFCCFBE
:1026700003C09EEF9093E800982F907609F0C6C0B3
:102680009E892F89188D91110CC0803829F4809172
:1026900040018093F10002C01092F1001092F1000D
:1026A00048C1422F50E0512B913051F4811141C16A
:1026B0004130510509F03DC1809140018D7F0BC033
:1026C000933061F4811135C14130510509F031C1B8
:1026D000809140018260809340012BC1953041F48C
:1026E0008091E80080FFFCCF20682093E30021C1A7
:1026F000963009F05FC0EB8CFC8C1092E9001092D0
:10270000730110927201123091F5109271011092C2
:1027100070010E941F1299E0BE016F5F7F4FDB01C5
:10272000E92F1D92EA95E9F799831A8391E09E8338
:1027300090EA98879AEF99872091720130917301FE
:10274000275F3F4F3C832B838D831092E9001092CB
:10275000730110927201F0927101E092700149E0F0
:1027600050E080E00E94B2100E941F12E2C0F0927E
:102770007101E09270010E94E31CDC011296ED9061
:10278000FC901397E114F10409F4C0C0D701ED9156
:10279000FC910480F581E02DBE016B5E7F4FC70187
:1027A0000995009719F00CF0C4C0C7C0F701E08488
:1027B000F184E8CF973009F4C0C0983021F481E06B
:1027C0008093F100B6C0993009F0B3C0837009F06E
:1027D000B4C0E7E1F1E081E021E036E390819923A4
:1027E00061F08093E9002093EB0091919093EC00CD
:1027F0003093ED008F5F873089F78EE78093EA0092
:102800001092EA008F898093760193C08B8D9C8D06
:102810001092E9001092730110927201909371016D
:1028200080937001898D811156C08E899D89913A5E
:1028300059F4813209F081C047E050E068E071E06E
:1028400080E00E94B21075C0913209F076C08332E8
:1028500089F4888D90E0982F88272F89822BA0E01B
:10286000B0E08093040190930501A0930601B0931A
:1028700007015FC0803269F48091E80082FFFCCFDD
:1028800067E088E091E00E94D9108BEF8093E80028
:1028900006C0823209F04DC08F8980930F0180916C
:1028A0003E01882319F0EEEFFAE002C0E0E0F8E024
:1028B0008091080190910901A0910A01B0910B014A
:1028C000803B9440A105B10509F07BC080910F01C8
:1028D00080FF93C076C00E94E31CDC0112960D912C
:1028E0001C9113970115110541F1D801ED91FC914F
:1028F0000190F081E02DBE016B5E7F4FC80109950C
:10290000811117C0F80100851185ECCF113009F451
:102910004EC0133091F48F89882309F445C082306A
:1029200081F440E867E089EA90E20E94E02288238F
:1029300021F08EEF8093E80079C081E28093EB0074
:1029400075C0813029F440E86BE08DE990E2EDCF6D
:10295000833099F70E94E31CDC011296ED90FC9005
:1029600013978E010F5F1F4F6801E114F10479F096
:10297000D701ED91FC910680F781E02DB801C701E8
:102980000995080F111DF701E084F184EECFD801FD
:102990001C92F60101900020E9F73197BF016C19F4
:1029A0007D0940E0C601C1CF67E870E202C06BE874
:1029B00070E26115710509F2FB01449150E080E875
:1029C00040CF0FB6F894A8958091600088618093FD
:1029D0006000109260000FBEA895EE3F2AE0F2075B
:1029E00039F08091FE0A9091FF0A91838083A1CFF4
:1029F0001092FF0A1092FE0A9CCFEE3F8AE0F80781
:102A000031F0808191819093FF0A8093FE0A87E7DD
:102A100097E7918380839BE088E10FB6F894A895AF
:102A2000809360000FBE9093600083CF6C960FB6CA
:102A3000F894DEBF0FBECDBFDF91CF91FF91EF9134
:102A4000BF91AF919F918F917F916F915F914F91C6
:102A50003F912F911F910F91FF90EF90DF90CF90BA
:102A60000F900FBE0F901F9018958F929F92AF926C
:102A7000BF92CF92DF92EF92FF926B017C010E9496
:102A80004C114B015C01C114D104E104F104F1F0DB
:102A90000E944C11DC01CB0188199909AA09BB09D4
:102AA000883E9340A105B10570F321E0C21AD10818
:102AB000E108F10888EE880E83E0981EA11CB11C85
:102AC000C114D104E104F10419F7DDCFFF90EF90B8
:102AD000DF90CF90BF90AF909F908F9008957F929E
:102AE0008F929F92AF92BF92CF92DF92EF92FF921E
:102AF0000F931F93CF93DF936C015B017A01809159
:102B00000F01882309F46BC080917601882309F4B2
:102B100066C080913F0180FF05C08091E000826027
:102B20008093E000E70110E00AEF83E0982E90E444
:102B3000792E2AE3822E209709F448C08FB7F894A3
:102B40009092E9009091E80095FF06C09091F20004
:102B5000272D291B922F01C090E08FBF91110AC031
:102B6000015009F43CC061E070E080E090E00E9418
:102B70003515E1CF292F30E0C217D3070CF49C2F75
:102B80008FB7F8949092E9002091E80025FF1CC0CF
:102B9000292F30E0C21BD30BF501915020F0419159
:102BA0004093F100FACFA20EB31E112319F08092C8
:102BB000E80009C09091E80095FD06C08092E80009
:102BC00011E0209709F010E08FBFB5CF1111B6CFFB
:102BD0005D9884E6809374011E141F0444F081E024
:102BE00090E0F6019383828380E090E001C0C7010A
:102BF000DF91CF911F910F91FF90EF90DF90CF90D9
:102C0000BF90AF909F908F907F9008951F920F92EA
:102C10000FB60F9211242F933F938F939F93AF93EF
:102C2000BF938091420190914301A0914401B091E2
:102C3000450130916B0123E0230F2D3720F40196DD
:102C4000A11DB11D05C026E8230F0296A11DB11DCF
:102C500020936B018093420190934301A093440120
:102C6000B093450180916C0190916D01A0916E012E
:102C7000B0916F010196A11DB11D80936C019093DD
:102C80006D01A0936E01B0936F01BF91AF919F91C1
:102C90008F913F912F910F900FBE0F901F9018951D
:102CA0001F920F920FB60F9211242F933F934F93C1
:102CB0005F936F937F938F939F93AF93BF93CF93C4
:102CC000DF93EF93FF9380916701882349F0809110
:102CD0006601811105C080916501882309F4ABC0AC
:102CE00080916101882309F4B6C080915D019091C3
:102CF0005E01A0915F01B0916001892B8A2B8B2B23
:102D000009F4A9C080915D0190915E01A0915F01DD
:102D1000B09160010197A109B10980935D01909381
:102D20005E01A0935F01B0936001892B8A2B8B2BEE
:102D300009F091C0D1E0E0915B01F0915C019F014D
:102D40002F5F3F4F30935C0120935B018491982F5C
:102D5000907FC82FCF70903821F48C2F0E94E811FB
:102D6000EACF9039F9F4E091C705F091C8050995CB
:102D70008D2780936501E0915B01F0915C01CF01AB
:102D8000019690935C0180935B01649180915A015C
:102D9000C81788F6C13009F058C0809159018111D7
:102DA000CACF53C097FD3AC03296F0935C01E093CE
:102DB0005B01F901249130E0382BA0916801B091BA
:102DC00069010E9462246C507E4F8F4F9F4F28EE06
:102DD00033E040E050E00E94402420935D013093B6
:102DE0005E0140935F015093600180915D0190917D
:102DF0005E01A0915F01B0916001892B8A2B8B2B22
:102E000051F581E090E0A0E0B0E080935D01909307
:102E10005E01A0935F01B09360011DC0903E29F454
:102E200010925C0110925B0186CF903F09F083CF36
:102E30001092610110C080916401E0916201F091F3
:102E400063019081892780834BCF67FD74CF8C2FDE
:102E50000E94711170CFFF91EF91DF91CF91BF91DF
:102E6000AF919F918F917F916F915F914F913F9122
:102E70002F910F900FBE0F901F9018951F920F92D9
:102E80000FB60F9211242F933F938F939F93AF937D
:102E9000BF93EF93FF9380916A01882309F44FC099
:102EA0008091550190915601A0915701B091580120
:102EB000892B8A2B8B2B51F180915401E091520187
:102EC000F0915301908189278083809155019091E1
:102ED0005601A0915701B0915801181619061A060B
:102EE0001B06D4F58091550190915601A091570190
:102EF000B09158010197A109B109809355019093B0
:102F00005601A0935701B093580126C01092660154
:102F100010926A0180916F008D7F80936F00909175
:102F20005401E0915201F09153018081282F30E04B
:102F3000892F90E080959095822393230CC08091F7
:102F40006501811109C080915401E0915201F09115
:102F50005301908189278083FF91EF91BF91AF91B9
:102F60009F918F913F912F910F900FBE0F901F90C7
:102F7000189590915A01923009F471C0292F30E0D0
:102F8000F901EC5EFE4F4081F901E05BFE4F80836A
:102F9000913031F420915001281302C090935901CF
:102FA0009F5F90935A0190E0FC01EA5AF04E249101
:102FB000FC01E95CF04E849130E0220F331FF901EF
:102FC000E75DF04E65917491F901E55EF04EA591D3
:102FD000B4919C91982B9C93413019F04330D9F0D7
:102FE000089590916400977F909364001092800000
:102FF000109281009091810098609093810090914F
:10300000810091609093810070935301609352010D
:1030100080935401089590916500977F9093650087
:10302000109290001092910090919100986090936E
:103030009100909191009160909391007093630141
:10304000609362018093640180915A01882321F08A
:103050006CE380E00E94711180E00C94E811089507
:103060002D9A0895BC0180E090E00C9435158FB145
:103070002CB193B130E02095309520743327A9010D
:1030800023E0559547952A95E1F7292F30E02095C3
:103090003095207133273595279535952795242B25
:1030A0008095807F822B089583B7817F83BF83B70C
:1030B000816083BF889583B78E7F83BF08958EBD5F
:1030C00000000DB407FEFDCF08952F923F924F925E
:1030D0005F926F927F928F929F92AF92BF92CF92A8
:1030E000DF92EF92FF920F931F93CF93DF93CDB7B1
:1030F000DEB72D970FB6F894DEBF0FBECDBFED82C1
:10310000E22EF12C9C012E0D3F1D37FD32C180387F
:1031100091050CF02EC19B01200F311D37FD29C1F7
:10312000603471050CF025C1DB0177FF04C0AA27CC
:10313000BB27A61BB70BA770BB279B0177FF02C05D
:10314000295F3F4F13E0359527951A95E1F777FFF3
:1031500008C02150310968E070E0FB01EA1BFB0B5D
:10316000DF01E02FE695E695E695CE2ED12C07708F
:1031700019F0FFEFCF1ADF0AB9017695762F66278F
:1031800077956795680F791F69587E4F8601020F02
:10319000131F19870887C12CD12CF8E0AF2EB12C52
:1031A00085010A1B1B0B1F830E83088519852017B9
:1031B000310709F4DEC02830310509F4DAC02F3FA9
:1031C0001FEF31070CF4CAC08B0100581F4F1D8739
:1031D0000C874B013B012B011C011C830B831A83C1
:1031E00009831B861A860A851B850E151F050CF0A0
:1031F000B5C010E82116310409F4B0C037FC89C00D
:103200002F3FEFEF3E0709F4B0C00A851B850C0D78
:103210001D1DFD81F13079F4F801E40FF51FE491F3
:10322000F0E08F010A2E01C0000F0A94EAF7F301C3
:10323000B0800B2925C0FD81F11114C0F801E40F05
:10324000F51FE491F0E00A2E02C0EE0FFF1F0A9472
:10325000E2F78F0100951095F401A080B12C0A21AE
:103260001B210EC0F801E40FF51FE491F0E08F017F
:103270000A2E01C0000F0A94EAF7F201B0800B2574
:103280000083109709F445C02730310509F441C087
:103290000A851B850C0D1D1DFD81F13089F4F80197
:1032A000E40FF51FE4910E2F10E00E8002C015957B
:1032B00007950A94E2F7EC85FD85B0800B2928C0BC
:1032C000FD81F11115C0F801E40FF51FE4910E2FF7
:1032D00010E00E8002C0159507950A94E2F700955C
:1032E0001095E981FA81A080B12C0A211B2110C020
:1032F000F801E40FF51FE4910E2F10E00E8002C0DC
:10330000159507950A94E2F7EB81FC81B0800B25B7
:1033100000830A851B850F5F1F4F1B870A870C855B
:103320001D850F5F1F4F1D870C8709811A810F5F55
:103330001F4F1A8309830B811C810F5F1F4F1C8352
:103340000B831FEF211A310AEFEF4E1A5E0AFFEFCF
:103350006F1A7F0A0FEF801A900A45CF2F5F3F4FF9
:1033600060587F4FCE0CDF1C20CF109709F090CF14
:10337000D0CF2D960FB6F894DEBF0FBECDBFDF9134
:10338000CF911F910F91FF90EF90DF90CF90BF9062
:10339000AF909F908F907F906F905F904F903F90F5
:1033A0002F90089560387105D0F440345105B8F479
:1033B000E3E1FAE180E1849FD001A0781124A60F17
:1033C0004770E40FF11DE491A958BE4F222319F074
:1033D0004C91E42B03C0E0954C91E423EC930895C9
:1033E0002F923F924F925F926F927F928F929F9215
:1033F000AF92BF92CF92DF92EF92FF920F931F9303
:10340000CF93DF93CDB7DEB729970FB6F894DEBF21
:103410000FBECDBFFC016A3069F4248D808D918D83
:1034200038E0239F800D911D1124918F808F178A82
:10343000168AAAC06D3009F4A7C099878887F48CD2
:10344000338C228C608C718C0689178900381105A9
:10345000C4F0A885B9855C962C915C97422F50E00A
:1034600056968D919C915797B6E02B9F800D911D9C
:103470001124E885F985978B868B258D21116EC0E7
:1034800083C0F0E46F16710424F7C80125E0F29EB2
:10349000800D911D112418161906DCF68F2D90E071
:1034A0009C838B83C301A8E0FA9E800D911D11249B
:1034B0001816190674F6B5E06B9FB0011124FB01D4
:1034C000E55EF54EFA83E98330E0888599850496B8
:1034D0009E838D83E981FA81E490353009F4E12CF3
:1034E000430188E0482EE0FC02C0532C01C0522C5E
:1034F00051100BC0321009C0E6944A948B819C8114
:10350000880E991E4110EFCF1BC068018C2D801BC7
:103510008F1590F754018A2D88198F1568F4252D81
:10352000A501B6018D819E813F830E94D2199FEF34
:10353000A91AB90A3F81EFCFAFEFCA1ADA0AE6CF6C
:103540003F5FEB81FC810E0F1F1F89819A810196DD
:103550009A838983363009F0BDCF7BCF6AEF64034D
:103560009001659F300D112420583F4F28173907CF
:103570005CF4A885B985ED91FC9111970190F081DB
:10358000E02D6AE0CD01099581E090E029960FB623
:10359000F894DEBF0FBECDBFDF91CF911F910F9189
:1035A000FF90EF90DF90CF90BF90AF909F908F9063
:1035B0007F906F905F904F903F902F900895109262
:1035C00049011092480184E1809301011092470162
:1035D0001092460181E08093030182E08093020112
:1035E00084E6809300010895CF939091D40593FDD4
:1035F0003CC09091D30593FF38C0C82F8091410102
:10360000882359F0E091C705F091C80509958823F2
:1036100021F080915A01823018F4C0934A0125C0EC
:1036200081E080936A0180914F01809366019091BF
:103630008100987F91609093810081E690EF909354
:103640008900809388008AE190E0A0E0B0E0809358
:10365000550190935601A0935701B0935801909152
:103660006F00926090936F00D8CFCF91089520E0C3
:1036700087E791E0B22FB111BFEFFC010024B193B5
:10368000B193B193B1930394D1F7089580917701E9
:103690008EBDE8E7F1E081910DB407FEFDCF8EBD50
:1036A00085E0E737F807B9F70DB407FEFDCF0895B9
:1036B000BF92CF92DF92EF92FF920F931F93CF931F
:1036C000DF939B01281B390B37FF03C031952195F0
:1036D0003109BB24B3942E3331054CF0B12C68175B
:1036E000790764F0A4E6B0E026E230E010C0DB0128
:1036F0009C0186E290E064E670E009C0382F292F33
:10370000CB01632F722FA6E2B0E024E630E0EB019C
:10371000C81BD90B8D01021B130B17FF03C011959A
:1037200001951109FE01D7FD3196F595E7952A1708
:103730003B071CF0EE24EA9402C0EE24E394A0E0E0
:10374000B0E050E00E2C000CFF086D01C80ED91E31
:103750006C157D059CF0BB2021F0A417B50724F063
:1037600010C0A417B50774F4E01BF10BF7FF04C0F9
:103770002E0D3F1DEC0FFD1F1196E7CF80E090E06E
:1037800001C0C901DF91CF911F910F91FF90EF9080
:10379000DF90CF90BF9008950F931F93CF93DF9347
:1037A0008C01C0E0D0E0F801EC0FFD1F64916623AE
:1037B00071F0E091CA05F091CB050190F081E02D08
:1037C0008AEC95E00995892B11F02196ECCFCE017A
:1037D000DF91CF911F910F9108958F929F92AF9299
:1037E000BF920F931F93CF93DF93CDB7DEB7A1970F
:1037F0000FB6F894DEBF0FBECDBF19A2423008F459
:103800004AE08E010F5D1F4F842E912CA12CB12C0C
:10381000A50194010E944024E62FB901CA0101507C
:103820001109EA3014F4E05D01C0E95CD801EC93C1
:10383000232B242B252B61F70115110571F0F801BD
:1038400001900020E9F73197AF01401B510BB801FF
:103850008AEC95E00E94E61002C080E090E0A1961C
:103860000FB6F894DEBF0FBECDBFDF91CF911F9191
:103870000F91BF90AF909F908F9008955F926F923D
:103880007F928F929F92AF92BF92CF92DF92EF92F0
:10389000FF920F931F93CF93DF93EC018B01CB012A
:1038A0008C1B9D0B97FF03C0919581959109552421
:1038B0005394CE9754F0512C0C171D076CF07E01D9
:1038C00084E690E0C6E2D0E00DC0C80104E610E056
:1038D00036E2E32EF12C06C078018E0186E290E0FC
:1038E000C4E6D0E038016E187F085C01AC1ABD0A4E
:1038F000B7FE03C0B194A194B108630177FE03C081
:103900002FEFC21AD20AD594C794C817D90714F05A
:103910008FEF01C081E0882E880F99080E151F05D2
:10392000C4F021E0552019F0A701BE0102C0AE018C
:10393000B7018EEC95E00E94D219CA18DB08D7FEB9
:1039400004C0C80DD91DC60CD71C8FEFE81AF80AA1
:10395000E5CFDF91CF911F910F91FF90EF90DF9016
:10396000CF90BF90AF909F908F907F906F905F901F
:103970000895FC0180917601811103C08FEF9FEFC4
:1039800008959FB7F89482E08093E9002091F200B7
:1039900030E01216130614F421E030E02115310551
:1039A00059F0289884E6809375018091F100808316
:1039B0008091F200882319F09FBFC90108958BE61A
:1039C0008093E800F9CF8091EC0581110DC082E071
:1039D0008093E80584E08093E9051092EB0510924E
:1039E000EA0581E08093EC0588EE95E008957894EF
:1039F00084B5826084BD84B5816084BD85B58260F4
:103A000085BD85B5816085BD80916E0081608093A4
:103A10006E0010928100809181008260809381000D
:103A2000809181008160809381008091800081601D
:103A300080938000809191008260809391008091BA
:103A400091008160809391008091900081608093CB
:103A500090008091C10084608093C1008091C1007A
:103A600082608093C1008091C10081608093C10019
:103A70008091C30081608093C3008091C000826008
:103A80008093C0008091C20081608093C2008091C9
:103A90007A00846080937A0080917A0082608093BB
:103AA0007A0080917A00816080937A0080917A0018
:103AB000806880937A0010927601109240011092F3
:103AC0003F018091D70081608093D70080EA809386
:103AD000D80089B5806189BD89B5826089BD09B486
:103AE00000FEFDCF61E070E080E090E00E943515BF
:103AF0008091D8008F7C80618093D8008091E00015
:103B0000807F8093E0008091E1008E7E8093E100D1
:103B10008DE08093E200559A209AEEEFFFE78591C1
:103B200094918B3F9C4D19F481E080933E0181EC90
:103B300080937C0085B1806F85B9249884B1866EAE
:103B400084B95E9A5F988AB1806D8AB9769A6E98C8
:103B500081B3806F81BB899880B38D7080BB80E515
:103B60008CBD81E08DBD85E090E00E9432185F9AA7
:103B700085E090E00E9432185E985C98CCE5D1E038
:103B80001C2F135FFE0184910E945F1821961C1365
:103B9000F9CF5C9A81E88093640081E080936500AE
:103BA000C0E0D4E080E00E945F182197D9F70E941E
:103BB000371887FF1FC05C9885EA0E945F185C9ADF
:103BC0002E982F982D9880916400806280936400D5
:103BD0000E945418FDCF2D980E943718847884389D
:103BE00071F00E9437188471843131F188EC90E0D3
:103BF0000E9432180E94371882FDEDCF3AC00E9411
:103C0000301888EC90E00E9432182F9882E090E003
:103C10000E94F8238F3F29F06FEF82E090E00E942E
:103C2000002484EF91E00E9432182F9A0E943718E6
:103C300084788438D9F3D5CF0E94301888EC90E08E
:103C40000E9432182E9882E090E00E94F823882388
:103C500029F060E082E090E00E94002484EF91E08F
:103C60000E9432182E9A0E94371884718431D9F339
:103C7000BDCF0E94301882E090E00E94F823882394
:103C800031F03E9A3F9A81E08093410104C0109246
:103C900041013E983F982E98CEEEDFEF0E943718F4
:103CA00086FF04C02E9A2F9A2D9A3BC0CC3F2FEF4F
:103CB000D20719F42E9A2F9805C0C831D10511F4F6
:103CC0002F9A2D980E94371BEE24E39400E128E5FB
:103CD0004CEA50E0BE0184E190E00E9465180E9429
:103CE000461B8BE190E00E943218C03F3FEFD307A4
:103CF00021F48AEF90E00E9432182196C931D10553
:103D000069F68CEB92E00E9432180E943018E09124
:103D1000CE05F091CF050190F081E02D8EEC95E07D
:103D2000099582E390E00E9432180E9437188111B1
:103D3000F8CF80E18093D5050E94461B85E00E9464
:103D4000B9178DE00E94B9178CED91E00E94F8231D
:103D500080934D018DED91E00E94F82380934E01F8
:103D600080914D0190914E01893E9D4F20F010921F
:103D70004E0110924D018FEF9FEF90938405809339
:103D800083050E94371B1092E3051092E205109202
:103D9000E1051092E00562E0462E512C612C712C59
:103DA00038ECC32ED12C48E8A42EB12C58EA252E8D
:103DB000312C2FB7F8948091420190914301A0914A
:103DC0004401B09145012FBF4091DA055091DB05C8
:103DD0006091DC057091DD052091DE05222341F024
:103DE0002091D605821B8093DF051092DE05DBC390
:103DF00084179507A607B70738F4481B423008F424
:103E0000D2C30E945418CFC321E02093DE058093D3
:103E1000D6059093D705A093D805B093D9052091E6
:103E2000D505820F911DA11DB11D8093DA059093D8
:103E3000DB05A093DC05B093DD058091D105909161
:103E4000D20501969093D2058093D1058091D30538
:103E50008093D4050E9437188093D3050E94371BA6
:103E60001092E3051092E2051092E1051092E00530
:103E700080914A01823009F473C0E8F4882311F17B
:103E8000813009F08EC30E94DF1A1092E105109272
:103E9000E0051092E3051092E205EE24E39400E4BD
:103EA00020E842ED54E160E070E080E090E00E94A4
:103EB000651882E074C3833009F47BC0843009F450
:103EC00034C36FC3EE24E39400E320E343EF58E1EF
:103ED00068E070E088E090E00E9465188BE490E074
:103EE0009093E1058093E00588E090E09093E305EE
:103EF0008093E2058AEE98E10E94CC1B87E590E072
:103F00009093E1058093E00582E190E09093E305D2
:103F10008093E20583EE98E10E94CC1B86E590E059
:103F20009093E1058093E00586E290E09093E305AD
:103F30008093E2058CED98E10E94CC1B84E490E034
:103F40009093E1058093E00581E390E09093E30591
:103F50008093E20582ED98E10E94CC1B81E01FC3B3
:103F60000E94DF1A2AE230E03093E1052093E00559
:103F700084E190E09093E3058093E20588EC94E17E
:103F80000E94CC1BE7E3F0E0F093E105E093E0054D
:103F90002EE130E03093E3052093E20560914D017E
:103FA00070914E0180E090E04AE00E94ED1B83E0BA
:103FB000F6C280910301882309F44CC040910201AC
:103FC0002091480130914901240F311D309349015E
:103FD000209348018091D40583FD04C09091D305BE
:103FE00093FD07C082FD16C08091D30582FF12C0E9
:103FF000E2C290914C019923A9F390914C0181E088
:10400000892780934C0180910101893218F48F5FD8
:1040100080930101C9016AE070E00E947124892B3C
:1040200071F4809146019091470101969093470168
:104030008093460180910101815080930101C90163
:1040400068EE73E00E947124873E934019F44F5F3D
:10405000409302018091010181111DC084E0809391
:104060004A01C0914601D091470180914D01909144
:104070004E018C179D0778F4D0934E01C0934D01EB
:104080008CED91E00E94F823C81729F06C2F8CED7D
:1040900091E00E940024C0914801D0914901CE01D5
:1040A0004296B6010E94712466277727681B790B18
:1040B000660F771F68537F4FF501E81BF90BCF019F
:1040C0000E943E1CCE018B96B6010E947124662789
:1040D0007727681B790B660F771F68537F4F950111
:1040E000281B390BC9010E943E1CCE018C5B9F4FDF
:1040F000B6010E94712466277727681B790B660F2B
:10410000771F68537F4FF501E81BF90BCF010E9421
:104110003E1CCE01835A9F4FB6010E947124662730
:104120007727681B790B660F771F68537F4F9501C0
:10413000281B390BC9010E943E1CCE018A589F4F93
:10414000B6010E94712466277727681B790B660FDA
:10415000771F68537F4FF501E81BF90BCF010E94D1
:104160003E1CCE0181579F4FB6010E9471246627E5
:104170007727681B790B660F771F68537F4F950170
:10418000281B390BC9010E943E1CCE0188559F4F48
:10419000B6010E94712466277727681B790B660F8A
:1041A000771F68537F4FF501E81BF90BCF010E9481
:1041B0003E1CCE018F539F4FB6010E94712466278B
:1041C0007727681B790B660F771F68537F4F950120
:1041D000281B390BC9010E943E1CCE0162E370E02E
:1041E0000E9471244C01EE24E3940AE222E34CE99C
:1041F00053E160E070E088279927881999090E94A7
:10420000651822E34CE953E160E070E082E390E05E
:10421000881999090E94651822E34CE953E160E08E
:1042200070E084E690E0881999090E94651822E3FD
:104230004CE953E160E070E086E990E08819990963
:104240000E946518CE01B1010E947124662777276C
:10425000681B790B660F771F6C557F4F47E02CE684
:1042600030E0F901E81BF90BCF010E94581B4C010B
:104270008C3E9F4F74F40E94EA23A30192010E9496
:104280000E2421E0672B682B692B09F420E0209392
:104290004B01C0914B0128EAC29FE0011124AE01FD
:1042A0004C555E4EEE24E39402E328E16CEF7FEF81
:1042B000C4010E946518AE014455504FE12C28E11D
:1042C0006CEF7FEFC4010E9465188091D105909139
:1042D000D2053AE0832E912CB4010E947124CB01C7
:1042E000C6E0D0E0BE010E94712417E8189FA0012B
:1042F000199F500D11244E57534F06E22BE16FE0EA
:1043000070E080E090E00E9465188091D105909166
:10431000D205B4010E947124CB01BE010E94712418
:10432000189FA001199F500D1124485A564FEE2492
:10433000E3942BE16FE070E080E090E00E9465186C
:104340000DE410E0C2E0D0E020E0AE01B8018EEC58
:1043500095E00E94D2192196CE30D105A9F70F5FC2
:104360001F4F0437110571F7EE24E3940CE027E2A8
:104370004AE059E062E070E08DE490E00E94651848
:1043800002E122E144ED58E060E070E08CE690E06C
:104390000E946518E12C22E14EE958E060E070E0EF
:1043A0008CE690E00E946518C09101018CE690E0D7
:1043B0004C018C1A9108EE24E39422E148E658E07F
:1043C00060E070E0C4010E946518E12C22E142E344
:1043D00058E060E070E0C4010E9465188091D1054A
:1043E0009091D2056CE370E00E94712433E0C39F8A
:1043F000E00111240A9790F4259708E124E346E9A7
:1044000057E060E270E0CE010E946518EE24E3946C
:1044100024E34AEF56E060E270E012C02A97E12CF4
:1044200008E124E34EE556E06EE170E0CE010E9423
:104430006518EE24E39424E342EC55E06EE170E06D
:10444000CE010E9465188091480190914901B10107
:104450000E94712466277727681B790B660F771FE8
:104460006C557F4F42E12CE630E0F901E81BF90B77
:10447000CF010E94581B01E710E0C5E3D0E020E027
:10448000AE01B8018EEC95E00E94D2192196CE3390
:10449000D105A9F70F5F1F4F0E37110571F7409136
:1044A0004C01FAE14F9FA001112442575A4FEE24CC
:1044B000E39409E02DE065E370E081E790E00E947D
:1044C000651802E010E0C2E0D0E020E0AE01B801E3
:1044D0008EEC95E00E94D2192196CE30D105A9F735
:1044E0000F5F1F4F0932110571F7EE24E3940CE0C2
:1044F00027E24AE059E062E070E082E090E00E944A
:10450000651884E090E09093E1058093E005909336
:10451000E3058093E205609146017091470180E0D8
:1045200090E04AE00E94ED1B3CC0EE24E39400E4DE
:1045300020E84EE851E060E070E080E090E00E940A
:10454000651883E891E00E94CC1B20914D013091C9
:104550004E0180914601909147012817390749F48F
:1045600082E791E00E94CC1B60914D0170914E0159
:1045700008C089E691E00E94CC1B609146017091D1
:10458000470180E090E04AE00E94ED1B809100012D
:10459000882321F081508093000103C080E00E94B5
:1045A000F41A0E94461B80E090E0892B09F401CCAC
:1045B0000E940000F5CB80914C0181112BCD1DCDC7
:1045C000CF92DF92EF92FF920F931F93CF93DF93DF
:1045D0001F92CDB7DEB7182F062FE42E862F880F37
:1045E0008E5F99830E94841083E00E948410F12ED4
:1045F000C12E9981D92E8C2D8F19801798F4F60130
:10460000E7FE02C0849101C080810E948410182FAF
:1046100080E00E9484108123FFEFCF1ADF0A81110E
:10462000EACF01C081E00F90DF91CF911F910F91F0
:10463000FF90EF90DF90CF9008950F931F93CF934B
:10464000DF938C0181E090E00E94F82380FF31C06D
:104650008AE090E00E94F8239FEF980F9E3F48F574
:1046600022E330E0D80157963C932E93569728E3E7
:1046700030E059963C932E935897CBE0D0E0D80188
:10468000ED91FC910190F081E02D682FC801099512
:10469000CE010E94F8232196C131D10581F70E94F5
:1046A000461B88EE93E0DF91CF911F910F910C9400
:1046B0003218DF91CF911F910F91089504970C94B8
:1046C0001D23E7E7F5E01382128288EE93E0A0E075
:1046D000B0E084839583A683B78381E291E09183E0
:1046E00080838FEF9FEF95878487EAECF5E0138254
:1046F00012821186128620E1238790878783108A91
:10470000118A128A138A148A81E391E0918380834B
:104710008BE391E095838483178A168A118E108E1D
:1047200081E0828F138E848F158E89E192E19093C0
:10473000C8058093C70508958F929F92AF92BF924C
:10474000CF92DF92EF92FF92CF93DF93EC016881DB
:1047500079818A819B81611571058105910521F41B
:1047600064E279ED8BE597E02DE133EF41E050E035
:104770000E940E2449015A019B01AC01A7EAB1E451
:104780000E942D246B017C01ACEEB4EFA5019401D5
:104790000E943B24DC01CB018C0D9D1DAE1DBF1D75
:1047A000B7FF03C00197A109B04888839983AA8302
:1047B000BB83BC01CD019F77DF91CF91FF90EF903C
:1047C000DF90CF90BF90AF909F908F9008950E9400
:1047D0009C23089580E191E00E949C2308956093BA
:1047E00010017093110180931201909313010895A9
:1047F000F999FECF92BD81BDF89A992780B50895A9
:10480000262FF999FECF1FBA92BD81BD20BD0FB6EC
:10481000F894FA9AF99A0FBE01960895052E97FB1F
:104820001EF400940E94252457FD07D00E944024C6
:1048300007FC03D04EF40C942524509540953095F8
:1048400021953F4F4F4F5F4F0895909580957095FC
:1048500061957F4F8F4F9F4F08950E946224A59FBF
:10486000900DB49F900DA49F800D911D112408956B
:10487000B7FF0C942D240E942D24821B930B0895C6
:10488000A1E21A2EAA1BBB1BFD010DC0AA1FBB1F54
:10489000EE1FFF1FA217B307E407F50720F0A21BC6
:1048A000B30BE40BF50B661F771F881F991F1A9433
:1048B00069F760957095809590959B01AC01BD015D
:1048C000CF010895A29FB001B39FC001A39F700DB7
:1048D000811D1124911DB29F700D811D1124911D08
:1048E0000895AA1BBB1B51E107C0AA1FBB1FA61737
:1048F000B70710F0A61BB70B881F991F5A95A9F789
:1049000080959095BC01CD010895EE0FFF1F059095
:10491000F491E02D099481E090E0F8940C949024B7
:04492000F894FFCF39
:1049240064140201FFFFFFFF00E10000000000002B
:1049340001000000030100C18081000000000000AC
:104944000011116F15321175125112271100000058
:0E49540000F019E6101D23FCFF00005E23009A
:00000001FF
